:10000000830100308A0068288C0003088301A60061
:100010002208A7002308A8009A30831281070B1139
:10002000990B3D28990A2128051E3D289901990A16
:100030003C28051E1F283A28160894000D15950126
:100040003D28150803191428013A031919280B3AF9
:1000500003191C280030051E0130A2000730A30040
:100060000310A20DA30B30282208A2000310160CC7
:100070002204960004309900950A970803194E2827
:1000800017080339031D4D288D1D86148D19861000
:100090008D1118188D150314980C97030F08031D64
:1000A0008F03FF309C07031C9D031D081C04031DC8
:1000B0005E28E1309C0001309D008D1483122708DA
:1000C000A2002808A300260883008C0E0C0E09004D
:1000D0000D3084000E3075200E30840022307520E3
:1000E0008301392A04068001840A0406031D72284C
:1000F0000034A400A51B832825088A002408A40A2C
:100100000319A50A82008313251883172408A40A5B
:10011000840000080800283463342934273430343C
:100120003034203442346F346234203442346C34FE
:10013000693463346B3400346C3463346434743441
:10014000653472346D342034763430342E343634A1
:1001500000348207003400340034003400340034AA
:1001600000340034003400340034003400340034EF
:10017000003400340034003400340034003482078A
:1001800041344234433444344534463447344834AB
:1001900049344A344B344C344D344E344F3450345B
:1001A00051345234533454348207613462346334EA
:1001B0006434653466346734683469346A346B3463
:1001C0006C346D346E346F34703471347234733413
:0201D000743485
:1002E6009F00803EA92901308312A921033081296C
:1002F6000D1D7B290D111408831208009F000A307A
:100306008F000F08031D84299F0B82298312080082
:10031600A0009708031D8C298D1120089800343001
:10032600970083120800A0291F08A5001E089E0A30
:1003360003199F0A79208312E1211F088312A50061
:100346001E0879200038031908009729A000831297
:1003560086110F3086052008F03986040615061129
:100366000F308605200EF039860406150611073073
:1003760086051B08F839860402308F000F0803191A
:100386000800C1298E03D22967308E00831273219B
:10039600DF291330C8295330C8292730C8290E0849
:1003A600133A0319CE292C3A0319CC296C3A0319AE
:1003B600D029AC3A0319C72983120800A00083127A
:1003C60086150F3086052008F039860406150611B5
:1003D6000F308605200EF039860406150611073003
:1003E60086051B08F839860402308F000F080319AA
:0A03F6000800F9298E0A0B2A403096
:100400008E000E0883127321182A1430002A5430EB
:10041000002A8E01012A0E08143A0319FF293C3ADA
:100420000319072A7C3A0319052A3C3A0319092AB9
:1004300083120800831286011F308316850086010F
:1004400095010D119901990AE1309C0001309D0040
:100450008D100A30900002309200143091000D107F
:100460009B018E0181129A30831281008B168B17AB
:10047000080083121A225A2276219C309E000030F6
:100480009F009621403073218B309E0000309F00EA
:100490009621FA308121FA30812176210D1D532ACF
:1004A00083127B21B6228D1C4E2A8D10831283224B
:1004B0002B234E2A83128611323081210F3086057C
:1004C0003030860406150611053081210615061107
:1004D00002308F000F08031D6A2A06150611053029
:1004E00081210F30860586160615061102308F0011
:1004F0000F08031D782A2830A9210830A9210C30C3
:10050000A9210630A929A10108309F0006309E00CC
:10051000A02A0730831286051F0886040A30A0002F
:10052000A00B902A0518A22AA10A8518A22AA10ABE
:100530000519A22AA10A8519A22AA10A03109F0D52
:100540009E0B892AF830831686000A30A000A00B83
:10055000A72A831206089A008316860107308312A1
:1005600086051B08F8398604210808009E000D1C2A
:10057000DD2A0D10D02A1E08831273211E088E005A
:10058000292B1E089B0083121E1CC82A0614080073
:10059000061008001E08E92A1E088312E121292BF3
:1005A0001308013A0319BB2A113A0319C12A023A66
:1005B0000319CA2A063A0319CC2A20301E02031C4A
:1005C000042B1B2B10308312F42A83127621FA2A73
:1005D00014308312A921292B10308312A921C5219F
:1005E0002030E121FD211030A921C521292B003027
:1005F000831273218E01292B1A0883128B21292B38
:100600000D141E089300292B1E08023A0319E22A32
:10061000013A0319E52A053A0319E82A0E3A0319A3
:10062000EC2A023A0319F72A073A0319F72A033A80
:100630000319FC2A002B80301E02031C252BA0303E
:100640001E020318252B07309E051E088312E12188
:10065000FD21831208009E00143A031D372B110858
:10066000143A031D352B9F01EA2B0230442B11084D
:10067000143A031D402B9F019F0A1E089100EA2B8C
:1006800090080319462B03309F00EA2B0430442BBB
:1006900000308A001108BF20922B920BFE2B0030F5
:1006A0008A001108BF20D32B1F08A20005302202A8
:1006B0000318FE2B03308A006130220703188A0AD0
:1006C0008200A72B482BB72BBE2B4D2B00308A0066
:1006D0001108BF20922B00308A001108D420B52BBE
:1006E0001F08A200053022020318FE2B03308A00E7
:1006F0007D30220703188A0A8200A72B662B6B2BFA
:10070000FE2BFE2B90080319B72B00308A0011082E
:10071000BF20B52B92080319FE2B920100308A00EE
:100720001108D42083128B21FE2B1F08A200053054
:1007300022020318FE2B03308A00A230220703187E
:100740008A0A8200A72BFE2B822BBE2B8A2B0A3013
:1007500090009201920AFE2B0A30D62B90080319C2
:10076000B72B00308A001108BF2083128B210A307A
:1007700090009201920A14309100FE2B9008031908
:10078000FE2B9003FE2B12080A3A031DCD2B0030DE
:100790008A001108D42083128B21920BFE2B00308B
:1007A0008A001108D42083128B2102309200FE2B84
:1007B0001F08A200053022020318FE2B03308A0016
:1007C000E530220703188A0A8200A72BAC2BAE2B38
:1007D000BE2BC32B00308A001108A920A2000430D0
:1007E00022020318BB2B03308A00FA3022070318B9
:1007F0008A0A8200542B702B952BD82B8312080069
:02400E00F13F80
:00000001FF
